:100000000BC018951895189518951895189518956A
:1000100018951895189518958FED8DBFC0ECE4EBE9
:100020004E2EDD275D2EEEE7F0E0A0E6B0E088275B
:100030008D933197E9F784B7082E877F84BF8FE1CE
:1000400081BD87E081BD5FD166248FEF8ABB8FE0E1
:1000500087BB80E08BBB80E088BB83E886B980E803
:1000600087B9EEE1F0E0A3E791E0A7D30091730038
:100070000E3C08F006C02DD185B78F7E806385BF0A
:10008000889580917300815080937300EEE1F0E0D9
:10009000A3E791E07BE780D38CE07DD11AD1ECED32
:1000A000F7E011D1E2E0F0E025D113D18FE711E0C4
:1000B0001FD100916E000A3008F003C0ECEEF7E0AB
:1000C00002D1ACE9B0E0EEE6F0E00ED3F4D0EEEE13
:1000D000F7E0F9D000916F000A3008F003C0E0EFBC
:1000E000F7E0F1D0ACE9B0E0EFE6F0E0FDD2E3D02C
:1000F0008FE716E0FDD0E2EFF7E0E5D08FEB12E0FE
:10010000F7D0ACE9B0E0E0E7F0E0EED2D4D0EEEE2C
:10011000F7E0D9D0A1E70D911C91043650E0150706
:1001200008F003C0E0EFF7E0CED0A1E70D911C91FD
:100130000A3050E0150708F003C0E0EFF7E0C3D045
:10014000ACE9B0E0E1E7F0E0C0D2B5D08FEB17E06A
:10015000CFD0E6EFF7E0B7D0A4E78C9187FB8827F4
:1001600080F9809580FBA4E78C9187F98C93A4E7B4
:100170008C9187FB0EF404C087E08093750003C068
:1001800089E18093750088EC90E031D1379A07B10E
:10019000007EA5E78C9190E0890F082707B936D13A
:1001A000A0E68D939C933798E0E6F0E0D190E08054
:1001B000FF24002796D1A2E6C5D1E8ECF7E066D28D
:1001C000E2E6F0E06AD1D0D1EDE0A2E6D7D2A4E732
:1001D0008C9187FB0EF432C0ECECF7E057D2E2E6EC
:1001E000F0E05BD1C1D1EDE0A2E6C8D2E2E6F0E0FA
:1001F00016D1AEE6DC92EEE6F0E0D080EE24FF24ED
:1002000000276FD1A6E69ED1E6E6F0E04BD1E2E60C
:10021000F0E043D1DAD1EDE0A2E6B0D2E0EDF7E0D4
:1002200035D2E2E6F0E039D19FD1EDE0A2E6A6D2E8
:10023000E2E6F0E0F4D0AFE6DC923CC0E4EDF7E0BB
:1002400025D2E2E6F0E029D18FD1EDE0AAE696D200
:10025000EAE6F0E0E4D0A0E7DC92E0E7F0E0D0806E
:10026000EE24FF2400273DD1A6E66CD1E6E6F0E0BF
:1002700019D1EAE6F0E011D1A8D1EDE0AAE67ED2EC
:10028000E8EDF7E003D2EAE6F0E007D16DD1EDE06A
:10029000AAE674D2EAE6F0E0C2D0A1E7DD92EC92E1
:1002A000A1E70D911C91013050E0150708F002C044
:1002B000A1E7F5D1FBCEACE9B0E08D91882311F038
:1002C00064D0FBCF0895DED1802D11F05ED0FBCF3E
:1002D000089581E060D014D080E85DC08FE72130C0
:1002E00039F08FEB223021F08FE8233009F08FECCA
:1002F000810F51C088EE93E07AD03197D9F70895F5
:1003000083E0992774C08AEF90E071D0B89AB99AC7
:10031000BA9ABB9AD49AD59ADD9885E090E067D0D6
:10032000DC98C098C198C29AC39ADC9AEF93FF9365
:10033000E5E1F0E050D0FF91EF91DC9855D0DC9AE8
:10034000EF93FF93E5E1F0E046D0FF91EF91DC9869
:100350004BD0DC9AEF93FF93E5E1F0E03CD0FF91C6
:10036000EF91DC9841D0C398DC9AEF93FF93E5E1DD
:10037000F0E031D0FF91EF91DC9836D088E20BD0DD
:100380008EE009D086E007D00895DD9A829505D0E9
:1003900004D02AD00895DD98F9CF859510F4C39A3A
:1003A00001C0C398859510F4C29A01C0C298859582
:1003B00010F4C19A01C0C198859510F4C09A01C08B
:1003C000C098DC9AEF93FF93E5E1F0E004D0FF9151
:1003D000EF91DC9808953197F1F70895689462F8E9
:1003E0000895E89462F8089581E090E000C0EF93EA
:1003F000FF93EE27E82BE92B31F0EAEFF0E031979D
:10040000F1F70197D1F7FF91EF910895369A369958
:10041000FECF369A3699FECF84B195B108953DD07E
:10042000992711278F2D880F80E8F82A802F881FA1
:1004300008F41FEF41F08F57082F07FD04C000326A
:1004400040F08FEF01C08827982FD82EE82EF82E85
:1004500009C08FE1801B082FF694E794D7949795F5
:100460000A95D1F7112351F09095D094E094F0942F
:1004700081E0980F8827D81EE81EF81E0F2DFE2C4D
:10048000ED2CD92E0895D094E094F09491E0D90EFB
:100490009927E91EF91E10950895D190E190F190E9
:1004A0000191089521913191419151910895102F19
:1004B00090E8FF0C001F0927990FF7941078652F1B
:1004C00090E8440F551F5927990F479560780038D9
:1004D0000895FF0C90E89027110F9795F794092F36
:1004E0000895102FBD2CDE2CEF2CF02E11234AF492
:1004F000B094D094E094F0949FEFB91AD90AE90A25
:10050000F90A0EE1FF2039F4FE2CED2CDB2CBB2484
:100510000850C2F723C032F00A95BB0CDD1CEE1C5C
:10052000FF1CF9CF01D0D5CFB7FE089590E8B916DA
:1005300011F4D0FE08959FEFD91AE90AF90A09F4D7
:1005400003950895DD92ED92FD920C9308959FE737
:10055000092FF92A9FEFD92EE92E0895DD24EE24E4
:10056000FF24002711270895A2DFC1F35038B1F30B
:100570001627005850580894051F12F418F4E7CFB6
:1005800008F0ECCF0AD0FF202AF0BB0CDD1CEE1CDB
:10059000FF1C9FCF0F5FDBF29CCF9F929924AA2470
:1005A000BB24992788E1990CAA1CBB1CDD1CEE1CFE
:1005B000FF1C30F4920EA31EB41ED91EE91EF91EB4
:1005C0008A9589F79F9008956DDF71DF503829F083
:1005D00090E869270CC00AF045D07BCF5FE3222763
:1005E0003327442701C05EDF62DF5038B1F30038A3
:1005F00099F3902F951B8BF312F434D0FACF9831E6
:1006000018F0222733274427983028F0232F342F3F
:1006100044279850F9CF992329F046953795279587
:100620009A95D9F7912F962742F014D0B0F6F79407
:10063000E794D7940F5F8BF68ACF10D051F008F46F
:1006400022DFFF2052F2DD0CEE1CFF1C0150CBF725
:100650007ECF84CFD20EE31EF41E0895D21AE30A91
:10066000F40A0895DF92EF92FF920F931F93D22E18
:10067000E32EF42E052F162F6F915F914F913F912E
:100680002F910895C895319600200895FBDF202D05
:10069000F9DF302DF7DF402DF5DF502D089582E092
:1006A00001C084E099279D938A95E9F70895000F8A
:1006B000111F221F331F0895009510952095309526
:1006C0000F5F1F4F2F4F3F4F0895019110810EC0B4
:1006D00001911191219130810BC00191108117FF7F
:1006E00005C03FEF2FEF04C00081112722273327D9
:1006F00037FF03C0E1DF8DE28D93CF93DF93CF927D
:10070000DF92EF92AA24BB24CC24DD24EE2440E225
:10071000CAE0DD2755E093E38881890F87FD9F704C
:1007200083FD907F891B89935A95A9F7C0DFAA1C86
:10073000BB1CCC1CDD1CEE1C4A9551F7E894EFE085
:10074000FF2782910ED0EB30E0F71EF068948A2DDF
:100750000CD088278D93EF90DF90CF90DF91CF91D1
:100760000895982F829501D0892F8F70805D26F093
:10077000803309F4089568948D93089594E08191ED
:100780008D939A95E1F70895E199FECFEEBB3196EE
:10079000089591E001C092E07B3751F47FB7F8945F
:1007A000F3DF8D918DBBE29AE19A9A95C9F77FBFED
:1007B0007727089591E001C092E0E6DFE09A8DB3DB
:1007C0008D939A95D1F708950000803EAA82113E3C
:1007D0000000C842363CBD3C00007A445757572EB3
:1007E0004156522E344D472E434F4D0020002E00CF
:0A07F00030002056000020410000F8
:00000001FF
